:100000007A2BFF3FFF3FFF3FA53003138312DA0037
:10001000DA0B0828000000000800073003138312E1
:10002000DA00DA0B1128080003138312AB0127084A
:1000300084000008D3000130D1002808D200510804
:10004000D000520803192828D00D5010FF3F222855
:100050005308D0055008D100520803193328D10C99
:10006000D113FF3F2D2851082A06031D61282908B6
:10007000003C03183F2804200420A9033728270840
:1000800084000008D3000130D1002808D2005108B4
:10009000D000520803195028D00D5010FF3F4A28B5
:1000A0005308D0055008D100520803195B28D10C21
:1000B000D113FF3F552851082A06031D6128FF3040
:1000C000AB002B08D0000800031383122008013A6C
:1000D000031D6C2887147E282008023A031D72280D
:1000E00087157E282008033A031D782807167E28E6
:1000F0002008043A031D7E2807147E283430DB00D4
:10010000FF30DA00DB0B85288828DA0B8528822867
:10011000CF30DA00DA0B8A28000087108711071227
:1001200007100330DC00FF30DB00FF30DA00DC0BAF
:100130009A28A128DB0B9D28A028DA0B9D289A2855
:1001400097280B30DB00FF30DA00DB0BA828AB2848
:10015000DA0BA828A5281830DA00DA0BAD28080039
:100160004030031383129F05F03083169F048312DF
:100170009F172708D000D00D5010D00D50105008F8
:100180009F041F140D209F1400309F180130D200CF
:100190005208013A031DCE280000C4281E08D200D0
:1001A000D3015208D300D2015208A8005308A90075
:1001B00083161E085204A8005308A9000030A904A1
:1001C00083121F102808D0002908D100080003134B
:1001D0008312DB01DA01D9018030D800DD01D11FA3
:1001E000F728D109D009D00A0319D10ADD0AD51F91
:1001F000FF28D509D409D40A0319D50ADD0AD10C80
:10020000D00C031C0C295408D90755080318550FA6
:10021000DA070318DB0A0310D01F14295408DA0781
:100220000318DB0A5508DB07DB0CDA0CD90CD80CF9
:10023000031CFF285D1C2729DB09DA09D909D80925
:10024000D80A0319D90A0319DA0A0319DB0A5B0869
:10025000D3005A08D2005908D1005808D00008002D
:10026000053003138312A7000530A8000A30A90047
:10027000AA0114205008FF3A031D4029871630298F
:1002800087120800053003138312A7000230A8006C
:100290000530A900AA0114205008FF3A031D802947
:1002A0000130A0000330DC00FF30DB00FF30DA005B
:1002B000DC0B5B296229DB0B5E296129DA0B5E29E5
:1002C0005B2958290B30DB00FF30DA00DB0B692992
:1002D0006C29DA0B692966291830DA00DA0B6E29E5
:1002E0000530A7000230A8000530A900AA0114209B
:1002F0005008FF3A031D7E290130A10064204229E5
:100300000800053003138312A7000130A800053050
:10031000A900AA0114205008FF3A031DBF2902308A
:10032000A0000330DC00FF30DB00FF30DA00DC0B24
:100330009A29A129DB0B9D29A029DA0B9D299A294D
:1003400097290B30DB00FF30DA00DB0BA829AB2943
:10035000DA0BA829A5291830DA00DA0BAD29053007
:10036000A7000130A8000530A900AA0114205008F8
:10037000FF3A031DBD290130A10064208129080036
:10038000053003138312A700A8010530A900AA01B4
:1003900014205008FF3A031DFC290330A00003304D
:1003A000DC00FF30DB00FF30DA00DC0BD829DF296E
:1003B000DB0BDB29DE29DA0BDB29D829D5290B3029
:1003C000DB00FF30DA00DB0BE629E929DA0BE6294E
:1003D000E3291830DA00DA0BEB290530A700A80171
:1003E0000530A900AA0114205008FF3A031DFA297C
:1003F0000130A1006420C0290800053003138312D6
:10040000A7000330A8000530A900AA011420500855
:10041000FF3A031D3B2A0430A0000330DC00FF300C
:10042000DB00FF30DA00DC0B162A1D2ADB0B192A51
:100430001C2ADA0B192A162A132A0B30DB00FF308C
:10044000DA00DB0B242A272ADA0B242A212A183087
:10045000DA00DA0B292A0530A7000330A80005309E
:10046000A900AA0114205008FF3A031D392A0130BF
:10047000A1006420FD290800053003138312A700A2
:100480000430A8000A30A900AA0114205008FF3A3D
:10049000031DCA2A0530A7000230A8000A30A900AF
:1004A000AA0114205008FF3AFF30031D0030A600B7
:1004B0000530A7000130A8000A30A900AA011420C5
:1004C0005008FF3AFF30031D0030D1005108A60448
:1004D0000530A700A8010A30A900AA01142050087D
:1004E000FF3AFF30031D0030D1005108A60405304B
:1004F000A7000330A8000A30A900AA011420500860
:10050000FF3AFF30031D0030D1005108A60405302A
:10051000A7000530A8000A30A900AA01142050083D
:10052000FF3AFF30031D0030D100510826040319A3
:10053000C92A87143430DB00FF30DA00DB0BA12A34
:10054000A42ADA0BA12A9E2ACF30DA00DA0BA62AD7
:10055000000087100330DC00FF30DB00FF30DA00E2
:10056000DC0BB32ABA2ADB0BB62AB92ADA0BB62A75
:10057000B32AB02A0B30DB00FF30DA00DB0BC12AD4
:10058000C42ADA0BC12ABE2A1830DA00DA0BC62ACE
:10059000A1013C2A0800031383122108013A031D1C
:1005A000792B0630A700B0205008A2005108A30004
:1005B0001E30D400D501E7205008A2005108A30046
:1005C0000130A400A50180302306D000803025062C
:1005D0005002031DED2A24082202031C782B02304E
:1005E000DB00FF30DA00DB0BF62AF92ADA0BF62AF9
:1005F000F32A4A30DA00DA0BFB2A0530A700023072
:10060000A8000A30A900AA0114205008FF3AFF30C0
:10061000031D0030A6000530A7000130A8000A30F5
:10062000A900AA0114205008FF3AFF30031D003032
:10063000D2005208A6040530A700A8010A30A9007C
:10064000AA0114205008FF3AFF30031D0030D200E9
:100650005208A6040530A7000330A8000A30A900FC
:10066000AA0114205008FF3AFF30031D0030D200C9
:100670005208A6040530A7000530A8000A30A900DA
:10068000AA0114205008FF3AFF30031D0030D200A9
:100690005208260403196C2BA1010330DC00FF3043
:1006A000DB00FF30DA00DC0B562B5D2BDB0B592B0C
:1006B0005C2BDA0B592B562B532B0B30DB00FF3006
:1006C000DA00DB0B642B672BDA0B642B612B183001
:1006D000DA00DA0B692B792B25082306031D722B10
:1006E000220824060319782BA40A0319A50AE32A71
:1006F000642008008B01073003138312990019301E
:100700009F00DF3083169F0040309100FF3085004E
:10071000FF3083128500043083168700831287011F
:100720008316811303138316302142218121C021B6
:10073000FD213C22CB22922B9C2BFF3FFF3FFF3F12
:10420000FF00FF00FF00FF00FF00FF00FF00FF00B6
:10421000FF00FF00FF00FF00FF00FF00FF00FF00A6
:10422000FF00FF00FF00FF00FF00FF00FF00FF0096
:10423000FF00FF00FF00FF00FF00FF00FF00FF0086
:10424000FF00FF00FF00FF00FF00FF00FF00FF0076
:10425000FF00FF00FF00FF00FF00FF00FF00FF0066
:10426000FF00FF00FF00FF00FF00FF00FF00FF0056
:10427000FF00FF00FF00FF00FF00FF00FF00FF0046
:10428000FF00FF00FF00FF00FF00FF00FF00FF0036
:10429000FF00FF00FF00FF00FF00FF00FF00FF0026
:1042A000FF00FF00FF00FF00FF00FF00FF00FF0016
:1042B000FF00FF00FF00FF00FF00FF00FF00FF0006
:1042C000FF00FF00FF00FF00FF00FF00FF00FF00F6
:1042D000FF00FF00FF00FF00FF00FF00FF00FF00E6
:1042E000FF00FF00FF00FF00FF00FF00FF00FF00D6
:1042F000FF00FF00FF00FF00FF00FF00FF00FF00C6
:10430000FF00FF00FF00FF00FF00FF00FF00FF00B5
:10431000FF00FF00FF00FF00FF00FF00FF00FF00A5
:10432000FF00FF00FF00FF00FF00FF00FF00FF0095
:10433000FF00FF00FF00FF00FF00FF00FF00FF0085
:10434000FF00FF00FF00FF00FF00FF00FF00FF0075
:10435000FF00FF00FF00FF00FF00FF00FF00FF0065
:10436000FF00FF00FF00FF00FF00FF00FF00FF0055
:10437000FF00FF00FF00FF00FF00FF00FF00FF0045
:10438000FF00FF00FF00FF00FF00FF00FF00FF0035
:10439000FF00FF00FF00FF00FF00FF00FF00FF0025
:1043A000FF00FF00FF00FF00FF00FF00FF00FF0015
:1043B000FF00FF00FF00FF00FF00FF00FF00FF0005
:1043C000FF00FF00FF00FF00FF00FF00FF00FF00F5
:1043D000FF00FF00FF00FF00FF00FF00FF00FF00E5
:1043E000FF00FF00FF00FF00FF00FF00FF00FF00D5
:1043F000FF00FF00FF00FF00FF00FF00FF00FF00C5
:02400E00443E2E
:00000001FF
